:020000040000FA
:040800007CEF05F094
:1008100003B23DEF04F0F2B458EF04F09EB060EF85
:1008200004F09EB268EF04F0F2A81AEF04F0F2B2FE
:100830001CEF04F05AEF05F0CD90F29207BC078E42
:10084000078C9EA029EF04F00101463F29EF04F038
:10085000472B07AE34EF04F0CECF51F1CFCF52F19A
:1008600046C153F147C154F1CF6ACE6A0101466BCC
:10087000476B9E90CD805AEF05F00392030103EE83
:1008800000F080517F0BE92604C0EFFF802B8151DF
:10089000805D700BD8A48B8200008051815D700B4D
:1008A000D8A48B9281518019D8B407905AEF05F0E3
:1008B000F2940101383F5AEF05F0392B5AEF05F059
:1008C0009E900101463F5AEF05F0472B5AEF05F085
:1008D0009E928B945BA16EEF04F08B94C3CF48F192
:1008E000C4CF49F1C28207B497EF04F03AC13EF198
:1008F0003BC13FF13CC140F13DC141F151C155F116
:1009000052C156F153C157F154C158F10101485138
:100910004E2749514F23E86A50230D2E97EF04F0DC
:100920004FC14AF150C14BF14E6B4F6B506B0201FE
:10093000002F5AEF05F03C0E006F05014E67A8EF3F
:1009400004F04F67A8EF04F05067A8EF04F0516778
:10095000ACEF04F0DCEF04F052C500F153C501F137
:1009600054C502F155C503F10101010E046F000EDB
:10097000056F000E066F000E076F7EEC17F000C1CA
:1009800052F501C153F502C154F503C155F5006795
:10099000D1EF04F00167D1EF04F00267D1EF04F06A
:1009A0000367DCEF04F04EC552F54FC553F550C553
:1009B00054F551C555F50E88050105015B6B2EB741
:1009C000E4EF04F05B818B8401015D67EFEF04F0DD
:1009D0005E67EFEF04F05F67EFEF04F06067F3EF3F
:1009E00004F023EF05F061C100F162C101F163C1C0
:1009F00002F164C103F10101010E046F000E056FE5
:100A0000000E066F000E076F7EEC17F000C161F15B
:100A100001C162F102C163F103C164F1006718EF23
:100A200005F0016718EF05F0026718EF05F003679E
:100A300023EF05F05DC161F15EC162F15FC163F159
:100A400060C164F10E80D57ED5BE32D0D6CF3AF1EA
:100A5000D7CF3BF138C13CF1E86AE8CF3DF1010165
:100A600047A73EEF05F0079C079E0101000E516F5E
:100A7000600E526F3D0E536F080E546F01013ABF66
:100A80004EEF05F03B674EEF05F03C674EEF05F08B
:100A90003D674EEF05F0F28853EF05F0F298516B89
:100AA000526B536B546BD76AD66A0101386B396B42
:100AB0005AEF05F002C0E0FF005001C0D8FF10005F
:100AC000A6B260EF05F00CC0A9FF0BC0A8FFA69E60
:100AD000A69CA684F29E550EA76EAA0EA76EA682AD
:100AE000F28EA694A6B272EF05F01200A96EA69E31
:100AF000A69CA680A8501200076A0E6A0F010E0E6F
:100B0000C16E860EC06E030EC26E0F01896A150E8D
:100B1000926E200E896E080E8A6EF30E936E8B6AAB
:100B2000900E946EF18E0D6A01014E6B4F6B506BFF
:100B30004A6B4B6B0F01280ED56EF28AB00ECD6E4C
:100B40009D800101516B526B536B546B556B566B0F
:100B5000576B586B596B5A6B5B6B5C6B079C079EB2
:100B6000760ECA6E9D8202013C0E006FCC6A160E94
:100B700076EC05F0E8CF00F1170E76EC05F0E8CF43
:100B800001F1180E76EC05F0E8CF02F1190E76ECC3
:100B900005F0E8CF03F1010103AFE9EF05F075ECD3
:100BA00018F0160E0C6E00C10BF060EC05F0170E7D
:100BB0000C6E01C10BF060EC05F0180E0C6E02C15A
:100BC0000BF060EC05F0190E0C6E03C10BF060EC3D
:100BD00005F000C15DF101C15EF102C15FF103C129
:100BE00060F100C161F101C162F102C163F103C1B1
:100BF00064F11A0E76EC05F0E8CF00F11B0E76ECEE
:100C000005F0E8CF01F11C0E76EC05F0E8CF02F11B
:100C10001D0E76EC05F0E8CF03F1010103AF3FEFC5
:100C200006F075EC18F01A0E0C6E00C10BF060ECBB
:100C300005F01B0E0C6E01C10BF060EC05F01C0EF4
:100C40000C6E02C10BF060EC05F01D0E0C6E03C1C2
:100C50000BF060EC05F01A0E76EC05F0E8CF00F131
:100C60001B0E76EC05F0E8CF01F11C0E76EC05F0DA
:100C7000E8CF02F11D0E76EC05F0E8CF03F100C1DC
:100C800065F101C166F102C167F103C168F1240E8B
:100C9000AC6E900EAB6E240EAC6E080EB86E000EED
:100CA000B06E1F0EAF6E0401806B816B0F01900E52
:100CB000AB6E0F019D8A0301806B816BA26B8B92DF
:100CC000898C400EC76E200EC66E0E94E1EC18F0B3
:100CD0008A840501006B016B026B036B046B056B6F
:100CE000066B0D6B0E6B0F6B106B116B126B196B30
:100CF0001A6B1B6B1C6B1D6B1E6B1F6B206B136BBE
:100D0000146B156B166B176B186BDFEC19F0200E5C
:100D100076EC05F0E8CF4EF5210E76EC05F0E8CF45
:100D20004FF5220E76EC05F0E8CF50F5230E76EC69
:100D300005F0E8CF51F54EC552F54FC553F550C5F6
:100D400054F551C555F5240E76EC05F0E8CF56F56F
:100D5000250E76EC05F0E8CF57F5260E76EC05F07B
:100D6000E8CF58F5270E76EC05F0E8CF59F50501E8
:100D70005B6B5C6B07900001F28EF28C07B02FEF7B
:100D800015F00EB074EF10F00EB848EF0AF0030142
:100D9000805181197F0BD8B42FEF15F013EE00F0BE
:100DA00081517F0BE126812BE7CFE8FFE00BD8B420
:100DB0002FEF15F023EE82F0A2511F0BD926E7CFBB
:100DC000DFFFA22BDF50780AD8A42FEF15F00780A1
:100DD00061C100F162C101F163C102F164C103F1BB
:100DE0000101040E046F000E056F000E066F000E69
:100DF000076F7EEC17F000AF07EF07F00101030E5D
:100E0000616F000E626F000E636F000E646F03016E
:100E10008251720AD8B474EF10F08251520AD8B4D9
:100E200074EF10F08251630AD8B4EFEF11F08251E1
:100E3000690AD8B449EF0EF082517A0AD8B45CEF4F
:100E40000FF08251490AD8B4E8EF0DF08251500AF0
:100E5000D8B406EF0DF08251700AD8B449EF0DF006
:100E60008251540AD8B474EF0DF08251740AD8B488
:100E7000BAEF0DF08251470AD8B46FEF0AF08251F1
:100E8000670AD8B48CEF0CF082514C0AD8B45EEFEC
:100E900007F024EF12F0040114EE00F080517F0BF4
:100EA000E12682C4E7FF802B12000D0E826F4BEC0F
:100EB00007F00A0E826F4BEC07F012008351300AE4
:100EC0003AE08351310AD8B4E9EF07F08351320A8E
:100ED000D8B469EF08F08351330AD8B477EF08F03B
:100EE0008351340AD8B485EF08F08351490AD8B445
:100EF000EFEF0BF08351500AD8B497EF0AF083510B
:100F0000700AD8B4E9EF0AF08351540AD8B423EF39
:100F10000BF08351740AD8B478EF0BF083514F0A69
:100F2000D8B4B5EF0BF083516F0AD8B4B5EF0BF01E
:100F3000D8A424EF12F06BEC1CF075EC18F02EC561
:100F400000F118EC18F004014C0E826F4BEC07F026
:100F50000401300E826F4BEC07F004012C0E826FFF
:100F60004BEC07F025C182F40401300E82274BECD4
:100F700007F026C182F40401300E82274BEC07F003
:100F800027C182F40401300E82274BEC07F00401E4
:100F90002C0E826F4BEC07F075EC18F02FC500F1AA
:100FA00018EC18F025C182F40401300E82274BECB6
:100FB00007F026C182F40401300E82274BEC07F0C3
:100FC00027C182F40401300E82274BEC07F06BEF4F
:100FD0000AF004014C0E826F4BEC07F00401310E55
:100FE000826F4BEC07F004012C0E826F4BEC07F084
:100FF000DFEC19F025C500F126C501F127C502F186
:1010000028C503F118EC18F022C182F40401300E57
:1010100082274BEC07F023C182F40401300E8227B3
:101020004BEC07F024C182F40401300E82274BEC14
:1010300007F025C182F40401300E82274BEC07F043
:1010400026C182F40401300E82274BEC07F027C141
:1010500082F40401300E82274BEC07F004012C0EC1
:10106000826F4BEC07F029C500F12AC501F12BC5B1
:1010700002F12CC503F118EC18F022C182F404012E
:10108000300E82274BEC07F023C182F40401300EAE
:1010900082274BEC07F024C182F40401300E822732
:1010A0004BEC07F025C182F40401300E82274BEC93
:1010B00007F026C182F40401300E82274BEC07F0C2
:1010C00027C182F40401300E82274BEC07F06BEF4E
:1010D0000AF004014C0E826F4BEC07F00401320E53
:1010E000826F4BEC07F04FEC1AF0F3EF07F00401BE
:1010F0004C0E826F4BEC07F00401330E826F4BEC09
:1011000007F098EC1AF0F3EF07F0B6EC18F084C390
:101110001EF185C31FF186C320F187C321F188C367
:1011200022F189C323F18AC324F18BC325F18CC337
:1011300026F18DC327F101011D6BC2EC18F03AECCA
:1011400018F0200E046F000E056F000E066F000EE3
:10115000076F8DEC17F000C121F501C122F502C126
:1011600023F503C124F53AEC1CF02EB3BFEF08F0D1
:101170000401530E826F4BEC07F0C4EF08F004013A
:101180004E0E826F4BEC07F004012C0E826F4BEC7D
:1011900007F02EB5D3EF08F00401570E826F4BEC29
:1011A00007F0D8EF08F00401450E826F4BEC07F012
:1011B00004012C0E826F4BEC07F02EB7E7EF08F01E
:1011C0000401560E826F4BEC07F0ECEF08F00401BF
:1011D000410E826F4BEC07F004012C0E826F4BEC3A
:1011E00007F075EC18F02FC500F130C501F131C5DD
:1011F00002F118EC18F022C182F40401300E8227AB
:101200004BEC07F023C182F40401300E82274BEC33
:1012100007F024C182F40401300E82274BEC07F062
:1012200025C182F40401300E82274BEC07F026C161
:1012300082F40401300E82274BEC07F027C182F4C0
:101240000401300E82274BEC07F004012C0E826F54
:101250004BEC07F075EC18F032C500F133C501F125
:1012600034C502F118EC18F022C182F40401300EEA
:1012700082274BEC07F023C182F40401300E822751
:101280004BEC07F024C182F40401300E82274BECB2
:1012900007F025C182F40401300E82274BEC07F0E1
:1012A00026C182F40401300E82274BEC07F027C1DF
:1012B00082F40401300E82274BEC07F004012C0E5F
:1012C000826F4BEC07F075EC18F035C500F136C5B0
:1012D00001F137C502F138C503F118EC18F020C14F
:1012E00082F40401300E82274BEC07F021C182F416
:1012F0000401300E82274BEC07F022C182F4040176
:10130000300E82274BEC07F023C182F40401300E2B
:1013100082274BEC07F004012E0E826F4BEC07F096
:1013200024C182F40401300E82274BEC07F025C162
:1013300082F40401300E82274BEC07F026C182F4C0
:101340000401300E82274BEC07F027C182F4040120
:10135000300E82274BEC07F004012C0E826F4BEC11
:1013600007F075EC18F039C500F13AC501F13BC53D
:1013700002F13CC503F118EC18F01FC182F404011E
:10138000300E82274BEC07F020C182F40401300EAE
:1013900082274BEC07F021C182F40401300E822732
:1013A0004BEC07F022C182F40401300E82274BEC93
:1013B00007F023C182F40401300E82274BEC07F0C2
:1013C00004012E0E826F4BEC07F024C182F404015D
:1013D000300E82274BEC07F025C182F40401300E59
:1013E00082274BEC07F026C182F40401300E8227DD
:1013F0004BEC07F027C182F40401300E82274BEC3E
:1014000007F004012C0E826F4BEC07F03DC500F194
:101410003EC501F13FC502F140C503F10101000ED7
:10142000046F000E056F010E066F000E076FACEC27
:1014300017F018EC18F01D6720EF0AF025EF0AF0FE
:1014400004012D0E826F4BEC07F024C182F40401DD
:10145000300E82274BEC07F025C182F40401300ED8
:1014600082274BEC07F004012E0E826F4BEC07F045
:1014700026C182F40401300E82274BEC07F027C10D
:1014800082F40401300E82274BEC07F06BEF0AF078
:101490000E980501566754EF0AF0576754EF0AF0AB
:1014A000586754EF0AF0596758EF0AF067EF0AF0EF
:1014B000D6EC0FF056C504F157C505F158C506F135
:1014C00059C507F17EEC17F003BFECEF11F098EC73
:1014D0001AF06BEF0AF055EC07F024EF12F023EE50
:1014E00082F0010EA26FA251D926DFCFA3F3A22B67
:1014F000780EA319D8B481EF0AF0F1EC18F073EF6D
:101500000AF00D0EA36FF1EC18F00A0EA36FF1ECC8
:1015100018F00401670E826F4BEC07F00401420ED5
:10152000826F4BEC07F055EC07F024EF12F004014A
:101530004C0E826F4BEC07F00401500E826F4BECA7
:1015400007F004012C0E826F4BEC07F084C31EF1F0
:1015500085C31FF186C320F187C321F188C322F11F
:1015600089C323F18AC324F18BC325F18CC326F1EF
:101570008DC327F10101C2EC18F03AEC18F0200EEF
:101580000C6E00C10BF060EC05F0210E0C6E01C179
:101590000BF060EC05F0220E0C6E02C10BF060EC5B
:1015A00005F0230E0C6E03C10BF060EC05F000C1DA
:1015B0004EF501C14FF502C150F503C151F500C10F
:1015C00052F501C153F502C154F503C155F5FEEFC3
:1015D0000BF004014C0E826F4BEC07F00401700E0F
:1015E000826F4BEC07F004012C0E826F4BEC07F07E
:1015F00084C31EF185C31FF186C320F187C321F187
:1016000088C322F189C323F18AC324F18BC325F156
:101610008CC326F18DC327F10101C2EC18F03AEC1E
:1016200018F000C14EF501C14FF502C150F503C1DC
:1016300051F500C152F501C153F502C154F503C182
:1016400055F5FEEF0BF004014C0E826F4BEC07F0EA
:101650000401540E826F4BEC07F004012C0E826FD4
:101660004BEC07F084C31EF185C31FF186C320F144
:1016700087C321F188C322F189C323F18AC324F1EE
:101680008BC325F18DC326F18EC327F10101C2EC76
:1016900018F03AEC18F00101000E046F000E056F0F
:1016A000010E066F000E076F8DEC17F0240E0C6E06
:1016B00000C10BF060EC05F0250E0C6E01C10BF0C3
:1016C00060EC05F0260E0C6E02C10BF060EC05F02C
:1016D000270E0C6E03C10BF060EC05F000C156F54F
:1016E00001C157F502C158F503C159F5FEEF0BF0E2
:1016F00004014C0E826F4BEC07F00401740E826FF4
:101700004BEC07F004012C0E826F4BEC07F084C306
:101710001EF185C31FF186C320F187C321F188C361
:1017200022F189C323F18AC324F18BC325F18DC330
:1017300026F18EC327F10101C2EC18F03AEC18F043
:101740000101000E046F000E056F010E066F000E02
:10175000076F8DEC17F000C156F501C157F502C1B6
:1017600058F503C159F5FEEF0BF004014C0E826FE2
:101770004BEC07F08351570A03E08351460A06E019
:10178000280E76EC05F0E890CAEF0BF0280E76EC08
:1017900005F0E880E8CF5AF583516F0A14E00401A0
:1017A0004F0E826F4BEC07F004012C0E826F4BEC56
:1017B00007F05AC5E8FF280E0C6EE8CF0BF060EC7E
:1017C00005F0EDEF0BF004016F0E826F4BEC07F0AC
:1017D00004012C0E826F4BEC07F0FEEF0BF00401BE
:1017E0004C0E826F4BEC07F00401490E826F4BECFC
:1017F00007F004012C0E826F4BEC07F0200E76EC04
:1018000005F0E8CF00F1210E76EC05F0E8CF01F10C
:10181000220E76EC05F0E8CF02F1230E76EC05F00F
:10182000E8CF03F118EC18F044EC16F00401730E45
:10183000826F4BEC07F004012C0E826F4BEC07F02B
:101840004EC500F14FC501F150C502F151C503F17C
:1018500018EC18F044EC16F00401730E826F4BEC98
:1018600007F004012C0E826F4BEC07F052C500F11B
:1018700053C501F154C502F155C503F118EC18F038
:1018800044EC16F00401730E826F4BEC07F0040178
:101890002C0E826F4BEC07F0240E76EC05F0E8CFAF
:1018A00000F1250E76EC05F0E8CF01F1260E76EC7E
:1018B00005F0E8CF02F1270E76EC05F0E8CF03F152
:1018C0003EEC12F004012C0E826F4BEC07F056C573
:1018D00000F157C501F158C502F159C503F13EECBD
:1018E00012F004012C0E826F4BEC07F0280E76EC00
:1018F00005F0E8B083EF0CF00401570E826F4BEC5B
:1019000007F088EF0CF00401460E826F4BEC07F0F5
:1019100055EC07F024EF12F08351300A1EE083519A
:10192000310A21E08351320A24E08351340A27E04E
:101930008351350A2AE08351360A2DE08351380A53
:1019400030E08351410A33E08351420A36E083514B
:10195000430A39E0D8A424EF12F00DC502F50EC5F4
:1019600003F5E9EF0CF00FC502F510C503F5E9EF3B
:101970000CF011C502F512C503F5E9EF0CF019C51D
:1019800002F51AC503F5E9EF0CF01BC502F51CC5FD
:1019900003F5E9EF0CF01DC502F51EC503F5E9EFEF
:1019A0000CF01FC502F520C503F5E9EF0CF013C5D7
:1019B00002F514C503F5E9EF0CF015C502F516C5DF
:1019C00003F5E9EF0CF017C502F518C503F5E9EFCB
:1019D0000CF026EE00F005010251D9260351D8B0D3
:1019E0000329DA26DFCFE8FF0A0A0CE0DFCF82F412
:1019F0004BEC07F00501032B023F0307030E03170F
:101A0000E9EF0CF055EC07F024EF12F083C31EF160
:101A100084C31FF185C320F186C321F187C322F15E
:101A200088C323F189C324F18AC325F18BC326F12E
:101A30008CC327F10101C2EC18F03AEC18F0160E35
:101A40000C6E00C10BF060EC05F0170E0C6E01C1BE
:101A50000BF060EC05F0180E0C6E02C10BF060ECA0
:101A600005F0190E0C6E03C10BF060EC05F000C11F
:101A70005DF101C15EF102C15FF103C160F100C11E
:101A800061F101C162F102C163F103C164F1E8EFE8
:101A90000DF083C31EF184C31FF185C320F186C3FB
:101AA00021F187C322F188C323F189C324F18AC3BA
:101AB00025F18BC326F18CC327F10101C2EC18F08C
:101AC0003AEC18F000C15DF101C15EF102C15FF1B5
:101AD00003C160F100C161F101C162F102C163F1B2
:101AE00003C164F1E8EF0DF083C31EF184C31FF15D
:101AF00085C320F186C321F187C322F188C323F176
:101B000089C324F18AC325F18CC326F18DC327F143
:101B10000101C2EC18F03AEC18F00101000E046F5C
:101B2000000E056F010E066F000E076F8DEC17F0AB
:101B30001A0E0C6E00C10BF060EC05F01B0E0C6E63
:101B400001C10BF060EC05F01C0E0C6E02C10BF035
:101B500060EC05F01D0E0C6E03C10BF060EC05F09F
:101B600000C165F101C166F102C167F103C168F10D
:101B7000E8EF0DF083C31EF184C31FF185C320F18C
:101B800086C321F187C322F188C323F189C324F1DD
:101B90008AC325F18CC326F18DC327F10101C2EC64
:101BA00018F03AEC18F00101000E046F000E056FFA
:101BB000010E066F000E076F8DEC17F000C165F186
:101BC00001C166F102C167F103C168F1E8EF0DF0F0
:101BD000160E76EC05F0E8CF00F1170E76EC05F066
:101BE000E8CF01F1180E76EC05F0E8CF02F1190EFE
:101BF00076EC05F0E8CF03F118EC18F044EC16F0A1
:101C00000401730E826F4BEC07F004012C0E826FFF
:101C10004BEC07F05DC100F15EC101F15FC102F163
:101C200060C103F118EC18F044EC16F00401730ED7
:101C3000826F4BEC07F004012C0E826F4BEC07F027
:101C40001A0E76EC05F0E8CF00F11B0E76EC05F0ED
:101C5000E8CF01F11C0E76EC05F0E8CF02F11D0E85
:101C600076EC05F0E8CF03F13EEC12F004012C0E07
:101C7000826F4BEC07F065C100F166C101F167C1ED
:101C800002F168C103F13EEC12F055EC07F024EFCD
:101C900012F00401690E826F4BEC07F004012C0E68
:101CA000826F4BEC07F00101040E006F000E016F14
:101CB000000E026F000E036F18EC18F020C182F4C2
:101CC0000401300E82274BEC07F021C182F404019D
:101CD000300E82274BEC07F022C182F40401300E53
:101CE00082274BEC07F023C182F40401300E8227D7
:101CF0004BEC07F024C182F40401300E82274BEC38
:101D000007F025C182F40401300E82274BEC07F066
:101D100026C182F40401300E82274BEC07F027C164
:101D200082F40401300E82274BEC07F004012C0EE4
:101D3000826F4BEC07F00101060E006F000E016F81
:101D4000000E026F000E036F18EC18F020C182F431
:101D50000401300E82274BEC07F021C182F404010C
:101D6000300E82274BEC07F022C182F40401300EC2
:101D700082274BEC07F023C182F40401300E822746
:101D80004BEC07F024C182F40401300E82274BECA7
:101D900007F025C182F40401300E82274BEC07F0D6
:101DA00026C182F40401300E82274BEC07F027C1D4
:101DB00082F40401300E82274BEC07F004012C0E54
:101DC000826F4BEC07F00101110E006F000E016FE6
:101DD000000E026F000E036F18EC18F020C182F4A1
:101DE0000401300E82274BEC07F021C182F404017C
:101DF000300E82274BEC07F022C182F40401300E32
:101E000082274BEC07F023C182F40401300E8227B5
:101E10004BEC07F024C182F40401300E82274BEC16
:101E200007F025C182F40401300E82274BEC07F045
:101E300026C182F40401300E82274BEC07F027C143
:101E400082F40401300E82274BEC07F004012C0EC3
:101E5000826F4BEC07F0200EF86EF76AF66A040109
:101E60000900F5CF82F44BEC07F00900F5CF82F4BE
:101E70004BEC07F00900F5CF82F44BEC07F00900BA
:101E8000F5CF82F44BEC07F00900F5CF82F44BEC70
:101E900007F00900F5CF82F44BEC07F00900F5CF0D
:101EA00082F44BEC07F00900F5CF82F44BEC07F01D
:101EB00055EC07F024EF12F08351630AD8A424EF05
:101EC00012F08451610AD8A424EF12F085516C0AF3
:101ED000D8A424EF12F08651410A42E08651440A08
:101EE0001BE08651420AD8B4C3EF0FF08651350A81
:101EF000D8B4ADEF13F08651360AD8B401EF14F020
:101F00008651370AD8B469EF14F08651380AD8B42C
:101F1000C7EF14F024EF12F00798079A04017A0E25
:101F2000826F4BEC07F00401780E826F4BEC07F0E8
:101F30000401640E826F4BEC07F081A8A7EF0FF04D
:101F40000401550E826F4BEC07F0ACEF0FF004016B
:101F50004C0E826F4BEC07F055EC07F024EF12F0BB
:101F60000788079A04017A0E826F4BEC07F0040190
:101F7000410E826F4BEC07F00401610E826F4BEC57
:101F800007F09DEF0FF00798078A04017A0E826F21
:101F90004BEC07F00401420E826F4BEC07F004019A
:101FA000610E826F4BEC07F09DEF0FF00101620EA6
:101FB000046F010E056F000E066F000E076F59C10A
:101FC00000F15AC101F15BC102F15CC103F17EEC89
:101FD00017F003BF33EF10F00E0E76EC05F0E8CFEC
:101FE0000CF10F0E76EC05F0E8CF0DF1100E76EC4B
:101FF00005F0E8CF0EF1110E76EC05F0E8CF0FF109
:10200000C7EC16F059C104F15AC105F15BC106F1E4
:102010005CC107F17EEC17F007828BEC16F0C7EC81
:1020200016F007928BEC16F059C100F15AC101F17C
:102030005BC102F15CC103F107928BEC16F0CC0E90
:10204000046FE00E056F870E066F050E076F7EECBE
:1020500017F000C10CF101C10DF102C10EF103C175
:102060000FF16BEF10F00101800E006F1A0E016F7F
:10207000060E026F000E036F42C104F143C105F169
:1020800044C106F145C107F17EEC17F003AF4CEFF8
:1020900010F075EC18F012000E0E76EC05F0E8CF9B
:1020A0000CF10F0E76EC05F0E8CF0DF1100E76EC8A
:1020B00005F0E8CF0EF1110E76EC05F0E8CF0FF148
:1020C00042C100F143C101F144C102F145C103F134
:1020D00007828BEC16F00CC100F10DC101F10EC1AD
:1020E00002F10FC103F112008251520A03E10E8284
:1020F0007BEF10F00E92078455C159F156C15AF189
:1021000057C15BF158C15CF13EC142F13FC143F19F
:1021100040C144F141C145F14AC14CF14BC14DF1BF
:1021200007940EA0B2EF10F0010165679FEF10F069
:1021300066679FEF10F067679FEF10F06867A3EF87
:1021400010F0B2EF10F0D6EC0FF065C104F166C1EB
:1021500005F167C106F168C107F17EEC17F003BF16
:10216000ECEF11F0D6EC0FF00101000E046F000E41
:10217000056F010E066F000E076FACEC17F004013F
:10218000720E826F4BEC07F004012C0E826F4BEC49
:1021900007F018EC18F01D67D3EF10F00401200EC3
:1021A000826FD6EF10F004012D0E826F4BEC07F01A
:1021B00024C182F40401300E82274BEC07F025C1C4
:1021C00082F40401300E82274BEC07F004012E0E3E
:1021D000826F4BEC07F026C182F40401300E822797
:1021E0004BEC07F027C182F40401300E82274BEC40
:1021F00007F004016D0E826F4BEC07F004012C0E0A
:10220000826F4BEC07F042C100F143C101F144C1C0
:1022100002F145C103F1010118EC18F044EC16F08D
:102220000401480E826F4BEC07F004017A0E826FB6
:102230004BEC07F004012C0E826F4BEC07F059C1F8
:1022400000F15AC101F15BC102F15CC103F101016E
:1022500018EC18F044EC16F00401630E826F4BEC9E
:1022600007F004012C0E826F4BEC07F059C100F10E
:102270005AC101F15BC102F15CC103F101010A0E17
:10228000046F000E056F000E066F000E076F8DECD9
:1022900017F0000E046F120E056F000E066F000E91
:1022A000076FACEC17F018EC18F01EC182F40401B3
:1022B000300E82274BEC07F01FC182F40401300E70
:1022C00082274BEC07F020C182F40401300E8227F4
:1022D0004BEC07F021C182F40401300E82274BEC55
:1022E00007F022C182F40401300E82274BEC07F084
:1022F00023C182F40401300E82274BEC07F024C185
:1023000082F40401300E82274BEC07F004012E0EFC
:10231000826F4BEC07F025C182F40401300E822756
:102320004BEC07F026C182F40401300E82274BECFF
:1023300007F027C182F40401300E82274BEC07F02E
:102340000401730E826F4BEC07F004012C0E826FB8
:102350004BEC07F075EC18F04CC100F14DC101F1E8
:102360004DEC13F00EB2B8EF11F00EA0EAEF11F041
:1023700004012C0E826F4BEC07F0200EF86EF76A0A
:10238000F66A04010900F5CF82F44BEC07F009006E
:10239000F5CF82F44BEC07F00900F5CF82F44BEC5B
:1023A00007F00900F5CF82F44BEC07F00900F5CFF8
:1023B00082F44BEC07F00900F5CF82F44BEC07F008
:1023C0000900F5CF82F44BEC07F00900F5CF82F459
:1023D0004BEC07F055EC07F00E9024EF12F00401DF
:1023E000630E826F4BEC07F004012C0E826F4BECF6
:1023F00007F029EC12F004012C0E826F4BEC07F071
:102400009CEC12F004012C0E826F4BEC07F018ECE0
:1024100013F004012C0E826F4BEC07F00101F80E53
:10242000006FCD0E016F660E026F030E036F3EEC60
:1024300012F004012C0E826F4BEC07F02EEC13F01F
:1024400055EC07F024EF12F00301A26B07902FEF79
:1024500015F0D8900E0E76EC05F0E8CF00F10F0ED7
:1024600076EC05F0E8CF01F1100E76EC05F0E8CF40
:1024700002F1110E76EC05F0E8CF03F10101000E38
:10248000046F000E056F010E066F000E076FACECB7
:1024900017F018EC18F01EC182F40401300E8227E8
:1024A0004BEC07F01FC182F40401300E82274BEC85
:1024B00007F020C182F40401300E82274BEC07F0B4
:1024C00021C182F40401300E82274BEC07F022C1B7
:1024D00082F40401300E82274BEC07F023C182F412
:1024E0000401300E82274BEC07F024C182F4040172
:1024F000300E82274BEC07F025C182F40401300E28
:1025000082274BEC07F004012E0E826F4BEC07F094
:1025100026C182F40401300E82274BEC07F027C15C
:1025200082F40401300E82274BEC07F004016D0E9B
:10253000826F4BEC07F01200120E76EC05F0E8CF3C
:1025400000F1130E76EC05F0E8CF01F1140E76ECF5
:1025500005F0E8CF02F1150E76EC05F0E8CF03F1B7
:1025600001010A0E046F000E056F000E066F000ECB
:10257000076F8DEC17F0000E046F120E056F000E42
:10258000066F000E076FACEC17F018EC18F01EC1C8
:1025900082F40401300E82274BEC07F01FC182F455
:1025A0000401300E82274BEC07F020C182F40401B5
:1025B000300E82274BEC07F021C182F40401300E6B
:1025C00082274BEC07F022C182F40401300E8227EF
:1025D0004BEC07F023C182F40401300E82274BEC50
:1025E00007F024C182F40401300E82274BEC07F07F
:1025F00004012E0E826F4BEC07F025C182F404011A
:10260000300E82274BEC07F026C182F40401300E15
:1026100082274BEC07F027C182F40401300E822799
:102620004BEC07F00401730E826F4BEC07F01200C5
:102630000A0E76EC05F0E8CF00F10B0E76EC05F013
:10264000E8CF01F10C0E76EC05F0E8CF02F10D0EAB
:1026500076EC05F0E8CF03F14DEF13F0060E76ECC3
:1026600005F0E8CF00F1070E76EC05F0E8CF01F1B8
:10267000080E76EC05F0E8CF02F1090E76EC05F0D5
:10268000E8CF03F14DEF13F0010175EC18F007846A
:102690004AC100F14BC101F107940101E80E046F3A
:1026A000800E056F000E066F000E076F8DEC17F0A1
:1026B000000E046F040E056F000E066F000E076F0C
:1026C000ACEC17F0880E046F130E056F000E066F4A
:1026D000000E076F7EEC17F00A0E046F000E056FF8
:1026E000000E066F000E076FACEC17F018EC18F038
:1026F00001011D6781EF13F00401200E826F84EF4A
:1027000013F004012D0E826F4BEC07F024C182F40C
:102710000401300E82274BEC07F025C182F404013E
:10272000300E82274BEC07F026C182F40401300EF4
:1027300082274BEC07F004012E0E826F4BEC07F062
:1027400027C182F40401300E82274BEC07F004010C
:10275000430E826F4BEC07F0120087C31EF188C353
:102760001FF189C320F18AC321F18BC322F18CC3ED
:1027700023F18DC324F18EC325F190C326F191C3BB
:1027800027F10101C2EC18F03AEC18F00101000E3B
:10279000046F000E056F010E066F000E076F8DECC3
:1027A00017F00E0E0C6E00C10BF060EC05F00F0E72
:1027B0000C6E01C10BF060EC05F0100E0C6E02C146
:1027C0000BF060EC05F0110E0C6E03C10BF060EC29
:1027D00005F004017A0E826F4BEC07F004012C0E19
:1027E000826F4BEC07F00401350E826F4BEC07F063
:1027F00004012C0E826F4BEC07F029EC12F0ACEFC9
:102800000FF087C31EF188C31FF189C320F18AC36B
:1028100021F18BC322F18CC323F18DC324F18EC32C
:1028200025F190C326F191C327F10101C2EC18F004
:102830003AEC18F0880E046F130E056F000E066F49
:10284000000E076F82EC17F0000E046F040E056F88
:10285000000E066F000E076F8DEC17F00101E80EF9
:10286000046F800E056F000E066F000E076FACEC54
:1028700017F00A0E0C6E00C10BF060EC05F00B0EA9
:102880000C6E01C10BF060EC05F00C0E0C6E02C179
:102890000BF060EC05F00D0E0C6E03C10BF060EC5C
:1028A00005F004017A0E826F4BEC07F004012C0E48
:1028B000826F4BEC07F00401360E826F4BEC07F091
:1028C00004012C0E826F4BEC07F018EC13F0ACEF08
:1028D0000FF087C31EF188C31FF189C320F18AC39B
:1028E00021F18BC322F18CC323F18DC324F18FC35B
:1028F00025F190C326F191C327F10101C2EC18F034
:102900003AEC18F0000E046F120E056F000E066F01
:10291000000E076F8DEC17F001010A0E046F000E18
:10292000056F000E066F000E076FACEC17F0120E6D
:102930000C6E00C10BF060EC05F0130E0C6E01C1C3
:102940000BF060EC05F0140E0C6E02C10BF060ECA5
:1029500005F0150E0C6E03C10BF060EC05F00401E0
:102960007A0E826F4BEC07F004012C0E826F4BEC59
:1029700007F00401370E826F4BEC07F004012C0EB8
:10298000826F4BEC07F09CEC12F0ACEF0FF087C3BA
:102990001EF188C31FF189C320F18AC321F18BC3C3
:1029A00022F18CC323F18DC324F18EC325F190C392
:1029B00026F191C327F10101C2EC18F03AEC18F0AE
:1029C000880E046F130E056F000E066F000E076F62
:1029D00082EC17F0000E046F040E056F000E066FF8
:1029E000000E076F8DEC17F00101E80E046F800EEA
:1029F000056F000E066F000E076FACEC17F0060EA9
:102A00000C6E00C10BF060EC05F0070E0C6E01C1FE
:102A10000BF060EC05F0080E0C6E02C10BF060ECE0
:102A200005F0090E0C6E03C10BF060EC05F004011B
:102A30007A0E826F4BEC07F004012C0E826F4BEC88
:102A400007F00401380E826F4BEC07F004012C0EE6
:102A5000826F4BEC07F02EEC13F0ACEF0FF081A877
:102A6000EDEF15F007A8A6EF15F00101800E006F3D
:102A70001A0E016F060E026F000E036F3EC104F1C5
:102A80003FC105F140C106F141C107F17EEC17F0ED
:102A900003BFEDEF15F03EEC16F03EC100F13FC173
:102AA00001F140C102F141C103F107828BEC16F044
:102AB0000CC104F10DC105F10EC106F10FC107F102
:102AC000F80E006FCD0E016F660E026F030E036FDE
:102AD0007EEC17F00E0E0C6E00C10BF060EC05F0F2
:102AE0000F0E0C6E01C10BF060EC05F0100E0C6EB9
:102AF00002C10BF060EC05F0110E0C6E03C10BF07F
:102B000060EC05F00784010175EC18F04AC100F192
:102B10004BC101F107940A0E0C6E00C10BF060EC82
:102B200005F00B0E0C6E01C10BF060EC05F00C0E05
:102B30000C6E02C10BF060EC05F00D0E0C6E03C1C3
:102B40000BF060EC05F00798EDEF15F007AAEDEF3C
:102B500015F00784010175EC18F04AC100F14BC172
:102B600001F10794060E0C6E00C10BF060EC05F04D
:102B7000070E0C6E01C10BF060EC05F0080E0C6E38
:102B800002C10BF060EC05F0090E0C6E03C10BF0F6
:102B900060EC05F0078455C100F156C101F157C141
:102BA00002F158C103F10794120E0C6E00C10BF034
:102BB00060EC05F0130E0C6E01C10BF060EC05F03B
:102BC000140E0C6E02C10BF060EC05F0150E0C6ECD
:102BD00003C10BF060EC05F0079A040180518119E4
:102BE0007F0B0BE09EA809D014EE00F081517F0B03
:102BF000E126E750812B0F01AD6E11EC19F080A496
:102C00000AEF16F0949C94928A84898CFC0ED31659
:102C100010EF16F0948C94828A94899C020ED31241
:102C2000BEEF06F00CC100F10DC101F10EC102F1C1
:102C30000FC103F1000E046F000E056F010E066F49
:102C4000000E076FACEC17F01DA13DEF16F014510C
:102C5000D8B43DEF16F00CC100F10DC101F10EC169
:102C600002F10FC103F1000E046F000E056F0A0E92
:102C7000066F000E076FACEC17F0120001010C6B31
:102C80000D6B0E6B0F6B12001EC182F40401300E2F
:102C900082274BEC07F01FC182F40401300E82271B
:102CA0004BEC07F020C182F40401300E82274BEC7C
:102CB00007F021C182F40401300E82274BEC07F0AB
:102CC00022C182F40401300E82274BEC07F023C1AD
:102CD00082F40401300E82274BEC07F024C182F409
:102CE0000401300E82274BEC07F025C182F4040169
:102CF000300E82274BEC07F026C182F40401300E1F
:102D000082274BEC07F027C182F40401300E8227A2
:102D10004BEC07F012000101005305E1015303E100
:102D2000025301E1002B4EEC17F075EC18F02C511A
:102D3000006F2D51016F420E046F4B0E056F000E98
:102D4000066F000E076F8DEC17F000C104F101C192
:102D500005F102C106F103C107F10CC100F10DC17B
:102D600001F10EC102F10FC103F107B2BCEF16F081
:102D700082EC17F0BEEF16F07EEC17F000C10CF1FC
:102D800001C10DF102C10EF103C10FF1120075EC8A
:102D900018F04CC100F14DC101F1060E76EC05F0C2
:102DA000E8CF04F1070E76EC05F0E8CF05F1080E48
:102DB00076EC05F0E8CF06F1090E76EC05F0E8CFE9
:102DC00007F17EEC17F000C118F101C119F102C141
:102DD0001AF103C11BF1290E046F000E056F000EDE
:102DE000066F000E076F8DEC17F0EE0E046F430EAA
:102DF000056F000E066F000E076F82EC17F018C10A
:102E000004F119C105F11AC106F11BC107F18DECDE
:102E100017F000C110F101C111F102C112F103C19B
:102E200013F1120E76EC05F0E8CF04F1130E76ECF8
:102E300005F0E8CF05F1140E76EC05F0E8CF06F1C9
:102E4000150E76EC05F0E8CF07F10D0E006F000EC1
:102E5000016F000E026F000E036F8DEC17F0180E5D
:102E6000046F000E056F000E066F000E076FACECCE
:102E700017F010C104F111C105F112C106F113C11F
:102E800007F182EC17F06A0E046F2A0E056F000E30
:102E9000066F000E076F7EEC17F01200BF0EFA6E81
:102EA000200E2D6F2C6BD890003701370237033777
:102EB000D8B05FEF17F02D2F54EF17F02C072D0728
:102EC0000353D8B412000331070B8009326F033962
:102ED0000F0B010F2C6F80EC5FF0336F2C0580EC33
:102EE0005FF0335D335F2C6B3233D8B02C272C333B
:102EF00032A974EF17F033512C2712009AEC18F016
:102F0000D8B0120003510719286F5DEC18F0D89063
:102F10000751031928AF800F1200286B81EC18F0BD
:102F2000D8A097EC18F0D8B012006CEC18F075EC43
:102F300018F01F0E296FADEC18F00B35D8B05DEC12
:102F400018F0D8A00335D8B01200292F9BEF17F046
:102F500028B184EC18F01200286B045105110611F9
:102F600007110008D8A081EC18F0D8A097EC18F051
:102F7000D8B01200086B096B0A6B0B6BADEC18F044
:102F80001F0E296FADEC18F007510B5DD8A4D5EFDB
:102F900017F006510A5DD8A4D5EF17F00551095D69
:102FA000D8A4D5EF17F00451085DD8A0E8EF17F0CA
:102FB0000451085F0551D8A0053D095F0651D8A00E
:102FC000063D0A5F0751D8A0073D0B5FD8900081EE
:102FD000292FC2EF17F028B184EC18F0286B81EC90
:102FE00018F0D890B1EC18F007510B5DD8A405EF9C
:102FF00018F006510A5DD8A405EF18F00551095DD7
:10300000D8A405EF18F00451085DD8A014EF18F00B
:10301000003F14EF18F0013F14EF18F0023F14EFD7
:1030200018F0032BD8B4120028B184EC18F0120069
:103030000101286B81EC18F0D8B01200B6EC18F042
:10304000200E296F003701370237033711EE27F0C2
:103050000A0E2A6FE7360A0EE75CD8B0E76EE55233
:103060002A2F2AEF18F0292F22EF18F028B11D81FE
:10307000D890120001010A0E286F200E296F11EE60
:103080001DF028512A6F0A0ED890E652D8B0E726D4
:10309000E7322A2F45EF18F00333023301330033B0
:1030A000292F3FEF18F0E750FF0FD8A00335D8B015
:1030B00012001DB184EC18F01200045100270551D4
:1030C000D8B0053D01270651D8B0063D022707516B
:1030D000D8B0073D032712000051086F0151096F56
:1030E00002510A6F03510B6F12000101006B016B5B
:1030F000026B036B12000101046B056B066B076B1F
:1031000012000335D8A012000351800B001F011FCD
:10311000021F031F003F94EF18F0013F94EF18F0D7
:10312000023F94EF18F0032B282B032512000735DC
:10313000D8A012000751800B041F051F061F071F90
:10314000043FAAEF18F0053FAAEF18F0063FAAEFD8
:1031500018F0072B282B07251200003701370237FC
:103160000337083709370A370B3712001D6B1E6B00
:103170001F6B206B216B226B236B246B256B266BE3
:10318000276B12001E510F0B1E6F1F510F0B1F6F6D
:1031900020510F0B206F21510F0B216F22510F0B6C
:1031A000226F23510F0B236F24510F0B246F2551D6
:1031B0000F0B256F26510F0B266F27510F0B276F13
:1031C00012008A969E96CC0EC96E9EA6E5EF18F068
:1031D0009E960B0EC96E9EA6EBEF18F08A860E84A3
:1031E00012008A969E96000EC96E9EA6F5EF18F004
:1031F0009E96000EC96E9EA6FBEF18F08A868A96F0
:103200009E96820EC96E9EA603EF19F09E96A3C3EA
:10321000C9FF9EA609EF19F081B20CEF19F08A865A
:10322000120081B2DDEF19F08A969E96000EC96EEB
:103230009EA618EF19F0C9AEDDEF19F09E96000EAC
:10324000C96E9EA621EF19F0C9CFE8FF240A07E155
:103250000E8600C504F501C505F50501066B0EA631
:103260005EEF19F005010651010A11E00651020A4C
:1032700012E00651030A13E00651040A14E0065155
:10328000050A15E00651090A16E05DEF19F0C9CFED
:1032900007F55DEF19F0C9CF08F55DEF19F0C9CF5B
:1032A00009F55DEF19F0C9CF0AF55DEF19F0C9CF47
:1032B0000BF55DEF19F0C9CF0CF5062BC9CFE8FF70
:1032C0000A0A6AE10E960751470A66E10951470A60
:1032D0000EE00951520A48E00951560A4DE00951E1
:1032E0004D0A50E009515A0A53E0CCEF19F00A5147
:1032F000470A16E00A514C0A19E00B51410A1CE03A
:103300000B51560A02E0CCEF19F00C51310A1AE0C9
:103310000C51320A1DE00C51330A20E0CCEF19F0B9
:1033200004C50DF505C50EF5CCEF19F004C50FF574
:1033300005C510F5CCEF19F004C511F505C512F55A
:10334000CCEF19F004C513F505C514F5CCEF19F051
:1033500004C515F505C516F5CCEF19F004C517F52C
:1033600005C518F5CCEF19F004C519F505C51AF512
:10337000E9EC1AF0CCEF19F004C51BF505C51CF5F6
:10338000CCEF19F004C51DF505C51EF5CCEF19F0FD
:1033900004C51FF505C520F526EE00F00501005116
:1033A000D9260151D8B00129DA26C9CFDFFF05019E
:1033B000012B003F0107030E01178A861200050149
:1033C000256B266B276B286B296B2A6B2B6B2C6B61
:1033D000216B226B236B246B899A9E96030EC96E18
:1033E0009EA6FED79E9623C5C9FF9EA6FED79E9693
:1033F00022C5C9FF9EA6FED79E9621C5C9FF9EA6DF
:10340000FED79E96C9529EA6FED7898AC950FF0A4A
:103410000AE121C529F522C52AF523C52BF524C5C6
:103420002CF51EEF1AF0200E2127E86A2223E86A05
:10343000232323A9ECEF19F04EEF1AF0899A9E96F8
:10344000030EC96E9EA6FED79E9623C5C9FF9EA6F3
:10345000FED79E9622C5C9FF9EA6FED79E9621C581
:10346000C9FF9EA6FED79E96C9529EA6FED7898A00
:10347000C950FF0A0AE021C525F522C526F523C556
:1034800027F524C528F54EEF1AF0200E2127E86A0B
:103490002223E86A232323A91EEF1AF01200899A37
:1034A0009E96060EC96E9EA6FED7898A899A9E961A
:1034B000C70EC96E9EA6FED7898A899A9E96050E6A
:1034C000C96E9EA6FED79E96C9529EA6FED7C9B0CB
:1034D00063EF1AF0898A1200899A9E96060EC96EC9
:1034E0009EA6FED7898A899A9E96200EC96E9EA6B0
:1034F000FED79E9602C1C9FF9EA6FED79E9601C129
:10350000C9FF9EA6FED79E9600C1C9FF9EA6FED704
:10351000898A899A9E96050EC96E9EA6FED79E96AA
:10352000C9529EA6FED7C9B08FEF1AF0898A120041
:1035300029C500F12AC501F12BC502F12CC503F103
:103540000101005105E101510F0BD8B46CEC1AF0E8
:103550000501FE0E2E6F0501200E2D6F899A9E9695
:10356000060EC96E9EA6FED7898A899A9E96020E7D
:10357000C96E9EA6FED79E962BC5C9FF9EA6FED7F6
:103580009E962AC5C9FF9EA6FED79E9629C5C9FF4D
:103590009EA6FED725EE2EF02D2F02D0D7EF1AF0E3
:1035A0009E96DECFC9FF9EA6FED7CCEF1AF0898A81
:1035B000899A9E96050EC96E9EA6FED79E96C95202
:1035C0009EA6FED7C9B0DEEF1AF0898A8EEC1CF0F9
:1035D000120019C502F51AC503F525EE5EF00501C6
:1035E0002D6B16EE00F005010251E1260351D8B013
:1035F0000329E226E7CFE8FF2C0A06E12DC5DEFF0E
:1036000005012D6B0CEF1BF0E7CFE8FF2A0A0CE059
:10361000E7CFDEFF05012D2B0501032B023F03073A
:10362000030E0317F1EF1AF005012E6B2F6B306BB1
:10363000316B326B336B346B356B366B376B386B8E
:10364000396B3A6B3B6B3C6B3D6B3E6B3F6B406B3E
:10365000416B426B436B446B456B466B476B486BEE
:10366000496B4A6B4B6B4C6B4D6BDDCFE8FF050133
:103670002D5105E0DDCFE8FF2D2F3AEF1BF00501BE
:10368000DDCF2DF52D5105E0DDCFE8FF2D2F44EFE7
:103690001BF00501DDCF2DF52D5105E0DDCFE8FF55
:1036A0002D2F4EEF1BF011EE27F00101B6EC18F0B4
:1036B0000501DDCF2DF52D5105E0DDCFE5FF2D2FE7
:1036C0005DEF1BF00101C2EC18F03AEC18F000C1FC
:1036D0002FF501C130F502C131F50501DDCF2DF522
:1036E0002D5105E0DDCFE8FF2D2F72EF1BF0050116
:1036F000DDCF2DF52D5105E0DDCFE8FF2D2F7CEF3F
:103700001BF00501DDCF2DF52D5107E0DDCFE8FFE2
:10371000E8A82E852D2F86EF1BF011EE27F0010172
:10372000B6EC18F00501DDCF2DF52D5114E0DDCFFD
:10373000E5FFDDCFE5FFDDCFE5FFDDCFE5FFDDCF49
:10374000E8FFDDCFE5FFDDCFE5FFDDCFE5FFDDCF36
:10375000E5FFDDCFE5FF0101C2EC18F03AEC18F00F
:1037600000C139F501C13AF502C13BF503C13CF591
:103770000501DDCF2DF52D5107E0DDCFE8FFE8A8ED
:103780002E832D2FBDEF1BF011EE27F00101B6ECBB
:1037900018F00501DDCF2DF52D5105E0DDCFE5FF5A
:1037A0002D2FCEEF1BF0010122C123F121C122F107
:1037B00020C121F11FC120F1C2EC18F03AEC18F041
:1037C00000C135F501C136F502C137F503C138F541
:1037D0000501DDCF2DF52D5107E0DDCFE8FF2D2FC1
:1037E000EDEF1BF0E8B02E8711EE27F00101B6ECEB
:1037F00018F0DDCFE8FFDDCFE8FFDDCFE8FFDDCF5C
:10380000E8FFDDCFE8FFDDCFE5FFDDCFE5FFDDCF72
:10381000E5FFDDCFE5FFDDCFE5FFDDCFE5FFC2EC66
:1038200018F03AEC18F000C132F501C133F502C1CD
:1038300034F5078455C159F156C15AF157C15BF1AE
:1038400058C15CF13EC142F13FC143F140C144F176
:1038500041C145F14AC14CF14BC14DF10794D6EC41
:103860000FF000C13DF501C13EF502C13FF503C1B6
:1038700040F5120021C500F122C501F123C502F176
:1038800024C503F1899A9E960B0EC96E9EA6FED79B
:103890009E9602C1C9FF9EA6FED79E9601C1C9FF92
:1038A0009EA6FED79E9600C1C9FF9EA6FED79E96F5
:1038B000C9529EA6FED725EE2EF00501200E2D6FD3
:1038C0009E96C9529EA6FED7C9CFDEFF2D2F60EF70
:1038D0001CF0898A1200899A9E96900EC96E9EA647
:1038E000FED79E96000EC96E9EA6FED79E96000E2F
:1038F000C96E9EA6FED79E96000EC96E9EA6FED7E6
:103900009E96C9529EA6FED7C9CF2EF59E96C95245
:103910009EA6FED7C9CF2FF5898A12000501200E79
:103920002927E86A2A23E86A2B232BA91200296B8E
:063930002A6B2B6B120054
:10BF0000E844F926000C160C2B0C3F0C520C640C68
:10BF1000760C860C960CA50CB30CC10CCF0CDC0C6B
:06BF2000E80CF40C000C1B
:00000001FF
